:10000000831600301C3085000030860083125C2887
:10001000051D11281108003A031D0F28080091033F
:1000200008001108003A031D08003B2080309100B1
:100030000800851D22281208003A031D2028080008
:10004000920308001208003A031D08004420803083
:1000500092000800051E33281308003A031D3128BA
:100060000800930308001308003A031D0800482005
:1000700080309300080040309B0086174E20861386
:100080004E209B0B3D2808003B2053203B200800BE
:100090003B2053203B2053203B20080030309A0067
:1000A0009A0B5028080001309C009A0B55289B0B96
:1000B00055289C0B55280800082019202A205C2868
:00000001FF
